:0A00060000308A00D22900000A1021
:100010008A100A1182070D340A34543449344534A5
:100020004D3450344F343D3400340A108A100A11D4
:1000300082070D340A342534753420345334453462
:10004000473455344E3444344F34533400340A105A
:100050008A100A1182070D340A3453343D34253492
:1000600064340034F701F801380803103918F70731
:10007000F70CF80CB918F707F70CF80C3919F70753
:10008000F70CF80CB919F707F70CF80C391AF70741
:10009000F70CF80CB91AF707F70CF80C391BF7072F
:1000A000F70CF80CB91BF707F70CF80C8A11B128FC
:1000B000B601B4010A30B500B301B20803196628CD
:1000C0003608B60A320784000008B70037082D3C0E
:1000D000031D73280130B4003608B60A32078400C5
:1000E0000008B7007D2837082B3C031D7D28360803
:1000F000B60A320784000008B70037082F3C0318FF
:100100000C293708393C031C0C293708303C031DE7
:10011000A0283208360784000008783C0319972885
:100120003208360784000008583C031DA028103010
:10013000B500B60A3608B60A320784000008B700D0
:1001400035080A3C031DBD2837082F3C0318BC287E
:100150003708393C031CBC280A30B8003308B90002
:100160003228303037027807B3003608B60A320733
:1001700084000008B700A4280C293508103C031D92
:100180000C293708603C0318CC2837087A3C031C3C
:10019000CC283708DF39CD283708B70037082F3C7F
:1001A0000318D6283708393C0318DE283708403CA6
:1001B00003180C293708463C031C0C2937082F3C30
:1001C0000318EF283708393C031CEF28330EB8001A
:1001D000F030B805303037023807B300F828330E56
:1001E000B800F030B805413037020A3E3807B30096
:1001F0003608B60A320784000008B7003708603CAA
:100200000318092937087A3C031C09293708DF3904
:100210000A293708B700CE28340B142935080A3CC0
:10022000031D1429B309B30A3308F8008A115D2AA3
:100230003608F8013502031820293508F7002C2963
:10024000F7010830B700B50DF70D3608770203182F
:10025000F700F80DB70B2329003478083208B500F1
:100260006430B60018217708B20078083030031DDA
:10027000402933184729B3194729331A2030422916
:10028000B3113312F80778080C1E4429990032087C
:10029000B5000A30B60018217708B200780830306F
:1002A000031D5629B3195B29331A2030F807780843
:1002B0000C1E582999003030B20732080C1E5E29F6
:1002C00099008A116C2A35308400000803197729B7
:1002D0000130F800F701F70B6B29F80B6A294A3057
:1002E000F700F70B712900000000800B68298A11C4
:1002F0008329B30132083302031887290430B4007C
:10030000FA30B5006329B40B8029B30A7A298A111F
:100310007E2A3308F700B31B9129341D9D29203014
:100320009629F709F70A7708B3002D30F800780806
:100330000C1E98299900341DB4153308B50064309B
:10034000B60018217708B30078083030031DAF29B4
:100350003418B629B419B629341A2030B129B41189
:100360003412F80778080C1EB32999003308B50039
:100370000A30B60018217708B30078083030031D22
:10038000C529B419CA29341A2030F80778080C1E78
:10039000C72999003030B30733080C1ECD299900C6
:1003A0008A119B2A84011F30830583161F08C039D8
:1003B0009F009B01073083129F00A0010130A10024
:1003C000A201A301A40119308316990026309800D8
:1003D0009030831298001E3083168500FF3086000F
:1003E00083128501831681130D3083120C1AFA29AA
:1003F0008316F52999000A300C1EFC2999004F300C
:100400000C1E002A99004B300C1E042A99003E3025
:100410000C1E082A99008C1E0B2A1A08A500250814
:100420000C1E102A99002508523C031D272A8C1EF9
:10043000172A1A08A60026080C1E1C2A990026084E
:10044000303C031905102608313C03190514250812
:10045000543C031D7F2AB20132080720B20AF7007C
:1004600077080C1E312A990009303202031D2C2A0C
:10047000A5012508043C031C562A273025078400C3
:100480008C1E402A1A0880002730250784000008A7
:100490000D3C0319562A2730250784000008B200B6
:1004A00032080C1E512A9900A50A392A273025073F
:1004B000840080012730B20058287808B1000D3040
:1004C0000C1E602A99000A300C1E642A990031081B
:1004D000B2001830B3002D290430B20032081520C4
:1004E000B20AF70077080C1E732A99000D30320209
:1004F000031D6E2A05143108B2007929051025085C
:10050000533C031D9B2A05081E39F7000310770C86
:10051000A600B20132082720B20AF70077080C1EA5
:100520008F2A990004303202031D8A2A2608B3005C
:0C0530001830B40089298316F4296300F8
:040000008A01032846
:00000001FF
